:10000000830100308A001628F50003088301BB0035
:100010008B1C0F2883120313A001A00A8B1003135B
:1000200083123B088300F50E750E09002030840012
:100030003630282083010730BA00FD30B900363051
:10004000840039302C208301D52D04068001840AD8
:100050000406031D25280034F00038208000840A9F
:1000600004087006031900342D2883120313B90005
:10007000BA1B43283A1B4B283A088A003908B90AA8
:100080000319BA0A820083133A1883173908B90A88
:06009000840000080800D6
:100A920083160313861083120800831603130616A7
:100AA20083120800830193018316141C552D8312AF
:100AB2001308080083160313141C612D0130622DE4
:100AC200003083120800F400F40AF403031900341E
:100AD2000310F00DF10DF20DF30D662D8301AD0043
:100AE20083169401831294012D089404141694160B
:100AF20008008301AB00A408031D822D2B083326B6
:100B0200842D2B08F725AC0008008301AF002F08C5
:100B12009300941BFF348316141C8C2D83128C11AA
:100B22000034831603130612861406168610941DCB
:100B3200982D83128C1D9A2D8C1108008301AC0014
:100B4200A408031DA82D2B08AD002C08B92D2B08D5
:100B5200AD002C081E2E83160313061286140616E9
:100B62008610941DB22D83128C1DB42D8C11080099
:100B72008301AE009225370825046226E5252E085A
:100B82006226E5252D086226E525C72D83018C11F5
:100B920083160612861006168614141ECE2D831294
:100BA2008C1DD02D8C1108000A26842600300519D0
:100BB2000130F000F10138067104031D2B27A00853
:100BC200031DCE26A127D72D8301AF0183168614DC
:100BD2000616EF2DAF0FEF2DFF30F52D831286187D
:100BE200EB2D831606120030831208008301AD003C
:0E0BF200861137082504013886250038031DBA
:100C0000FA2D2D0886250038031D012E5325AE0030
:100C1000861508007030831603138F0081120115AA
:100C20008114011406309F00051085100515061467
:100C3000861101130B168B17831208008301AE0077
:100C400086113708250486250038031D212E2E081D
:100C500086250038031D272E2D0886250038031D04
:100C60002C2E861508008301AD0092253708250437
:100C70006226E5252D086226E525AC2537082504E2
:100C800001386226E5254926AE004E25C7252E08E7
:100C900008008301B001AF018316061600308312ED
:100CA000861801303007F0007007B0008316061276
:100CB0008312AF0A08302F02031C4C2E0310B00C15
:100CC000300808008301AF00831606128312B001BA
:100CD0003008F0002F08F200F301F00A722E031022
:100CE000F20DF30DF00B6F2EF21F792E8316861482
:100CF0007B2E83168610061606128312B00A083061
:100D0000300203180034682E0030F8260F30AB0094
:100D10000C309F254030AB000A309F25FF30AB00E0
:100D200000309F25FF30AB0001309F250130F826B1
:100D30000F30AB000C309F254030AB000B309F25AF
:100D4000FF30AB0000309F25FF30AB0001309F2DFE
:100D50008301AE003F3083169405831294012E0860
:100D600094042D0883169404C22E8316141783123C
:100D70001412CC2E83161417BF2E8316141383124D
:100D80001416CC2E83122C080319B52E023A03191F
:100D9000BA2E013A0319BD2E9416080010307A2598
:100DA0000F39AA00E92EA8010C30A9002A08A100D9
:100DB000A201A601A701F62EFE30E32EAA30A8005C
:100DC0000A30E52EC030A8000F30A9002A08A10083
:100DD000F62E2A08073A0319E22E0C3A0319DE2EE2
:100DE000063A0319DC2E033A0319D32EA00108009A
:100DF0008301AB009412AB08031D112FC030AC006F
:100E00000A306F2514163608831693008312861055
:100E10000612831686140616831285100514A40183
:100E200008002B0B0800230B182F0330AC001C2FDD
:100E3000A308031D1F2FAC01AD010130A8268316A6
:100E40008611061186140612831286150510851464
:100E5000A401A40A08000030830105190130B8007C
:100E6000A101A801A901051D472F0130F826AB01FA
:100E700004309F2512307A25AA00FF30AB000030E5
:100E80009F25FF30AB0001309F250030582F0030E8
:100E9000F826AB0104309F2512307A25AA00FF30D6
:100EA000AB0000309F25FF30AB0001309F250130A3
:100EB000F8260F30AB0004309F250F30AB00003018
:100EC0009F25AB0101309F2D83012A08F0002B08DC
:100ED000F1002C08F2002D08F3000330642570089F
:100EE000AE007108AF007208B0007308B100503056
:100EF00081000B11B201B301B401B5018B2F0B1DA1
:100F00007F2F0B1183120313B20A0319B30A0319BB
:100F1000B40A0319B50A3508803AF0003108803A5E
:100F20007002031D9D2F30083402031D9D2F2F08D2
:100F30003302031D9D2F2E083202031C7F2F8301D5
:100F400008008301280EF039AB0012309F252908D4
:100F5000F1002808F000F030F0050F30F105043002
:100F6000F2000310F10CF00CF20BB12F7008AB0083
:100F700013309F25EF2F003027020A300319260275
:100F8000031CC52FA209A601A701A208031003197B
:100F9000CC2FA80DA90DCE2FA90CA80CA60A0319B9
:100FA000A70ADE2F0310A80DA90D2908C03A2804AE
:100FB000031DDE2FFE30A8000F30A9004B30E32FB9
:100FC000A809A909C830AA00AB01EC2FA809A909F2
:100FD000F430AA000130AB00AC01AD01642F210850
:100FE000073A0319E02F0C3A0319E02F063A0319C8
:100FF000D22F033A0319BB2FE62F7D344034FF3440
:02400E00703F01
:00000001FF
